:020000040000FA
:06000000C93001303A286E
:08000800A000030EA100831209
:1000100005191128831601178312B2308100B1012E
:100020002C2883160113831203140B190310A80D37
:10003000A90DAA0DAB0DAC0DAC16FF302C02031DA3
:100040002C28FA302B02031D2C2832152A08AF0069
:100050002908AE002808AD008B100B11210E83007B
:06006000A00E200E0900B5
:04006600003400342E
:0C007400203084008001840A80300402E7
:10008000031C3C28DA2183160C3085058701831276
:10009000850187010730990000309A0010308316DF
:1000A0008E008312603083168F0083120030831617
:1000B00091009F008312C830831681008312313073
:1000C0009000003083168C00831210308B00BD1B13
:1000D0006F2885196F286400851D6B28E122C822CE
:1000E00081018E018F010B118B100B108C018B176E
:1000F000872032199320B40B852803108519031427
:10010000BA0DF0303A0203193C2127237828640005
:100110003310B10A311F9228AC01AB01AA01A90129
:10012000A801B101080032110130B7008B13203053
:10013000370783169B001C141A088312A400103082
:10014000370783169B001C141A088312A300A6000D
:100150000230A6060030370783169B001C141A08CD
:100160008312A200A7000130A7068B17331CBE28FC
:1001700022090339A200A309A409A50924082F0212
:10018000031D362923082E02031D362922082D02BD
:10019000031D362901303702031DD3283E18D3280A
:1001A0003E143F14FC2102303702031DDC28BE1828
:1001B000DC28BE143F140B2203303702031DE52850
:1001C0003E19E5283E153F14172204303702031D5F
:1001D000EE28BE19EE28BE153F1423220530370243
:1001E000031DF7283E1AF7283E163F143222063028
:1001F0003702031D0029BE1A0029BE163F143E22F5
:1002000007303702031D09293E1B09293E173F14F9
:100210004A2208303702031D1229BE1B1229BE17BD
:100220003F14552209303702031D1B295E181B2974
:100230005E143F1460220A303702031D2429DE18A1
:100240002429DE143F146B220B303702031D2D29A5
:100250005E192D295E153F1476220C303702031DDE
:100260003629DE193629DE153F148122B70A0D30F2
:1002700037020318080096280130B600B400B50014
:10028000B70085018701B2138720B40B54290310EE
:1002900085190314BA0DF0303A0203197C29B50B05
:1002A00054299630B5008621321D44293211331C61
:1002B0005E292D090339AD00AE09AF092F1C442971
:1002C0002D083002031944292D08B0002E1E4429A0
:1002D0008B1320303707BC002F08BB00C52110301E
:1002E0003707BC002E08BB00C52100303707BC0013
:1002F0002D08BB00C5218B1785018701B70AB60100
:100300000D303702031C4429C8220800013037028F
:1003100003198C220230370203199122033037026D
:10032000031996220430370203199B220530370245
:100330000319A022063037020319A522073037021D
:100340000319AA22083037020319AF2209303702F5
:100350000319B4220A3037020319B9220B303702CD
:100360000319BE220C3037020319C32208003F1CB8
:1003700008003F101030BC003E08BB00C5213030E3
:10038000BC005E08BB00C52108008B133B08831628
:100390001C159A0083123C0883169B0055309D0063
:1003A000AA309D009C1464009C18D3291C11831250
:1003B0008B170800831600309B001C141A08831248
:1003C000BD00831610309B001C141A088312BE0057
:1003D000831630309B001C141A088312DE00FF3095
:1003E000C800CA15CB15CC15CD15CE15CF15D01517
:1003F000D115D215D3150800C130BE05FF30DE057A
:100400000130C405C0000030C200C600BD185F1432
:10041000BD18DF140800C230BE05FF30DE05023013
:10042000C405C0000030C200C6005F100800C43020
:10043000BE05FF30DE050630C405C0000030C20036
:10044000C6005F100800C830BE05FF30DE0518305A
:10045000C405C0000030C200C600BD185F14BD183E
:10046000DF140800D030BE05FF30DE052230C405A1
:10047000C0000030C200C6005F100800E030BE05BA
:10048000FF30DE052630C405C0000030C200C600C3
:100490005F1008007F30BE05C030DE05C030C505E6
:1004A000C1000030C300C7000800BF30BE05C03027
:1004B000DE053030C505C1000030C300C7000800AC
:1004C0003F30BE05C130DE059030C505C1000030AB
:1004D000C300C70008003F30BE05C230DE05C03093
:1004E000C505C1000030C300C70008003F30BE058D
:1004F000C430DE053030C505C1000030C300C70080
:1005000008003F30BE05C830DE059030C505C1008B
:100510000030C300C7000800103085060030870691
:100520000800203085060030870608002130850647
:100530000030870608000230850602308706080072
:1005400020308506043087060800213085060430F7
:10055000870608000030850618308706080000303E
:100560008506213087060800003085060930870699
:100570000800003085061830870608000030850620
:1005800021308706080000308506093087060800FC
:100590003E18FC21BE180B223E191722BE19232239
:1005A0003E1A3222BE1A3E223E1B4A22BE1B552252
:1005B0005E186022DE186B225E197622DE19812217
:1005C0000800B601B401B5013D1CE92ABD01BD1406
:1005D000EB2ABD013D143D08B6006400EF2AF02A65
:1005E000F12AF22AF32AFF30B51B8500B51F8501D9
:1005F000B40BED2AB50BED2A0310B60CB608031D9B
:10060000ED2A0030BC003D08BB00C52108000512E2
:100610005C180516DC1C8512DC1885165C1D05109F
:100620005C190514DC1D8510DC1985145C1E87100F
:100630005C1A8714DC1E0711DC1A07155C1F0710F3
:100640005C1B0714DC1F8712DC1B871608008F0851
:10065000031908008F0178308E00C80F592DC80A81
:10066000441C572B461C482BCA1C392BCA014A155F
:10067000652B4A1D3E2BCA01CA15652BCA1D432B8B
:10068000CA014A16652B4A1E652BCA01CA14652B7E
:100690004A1D4D2BCA014A16652BCA1D522BCA0191
:1006A0004A16652B4A1E652BCA01CA14652BCA1C43
:1006B0005C2BCA014A15652B4A1D612BCA01CA155C
:1006C000652B4A1E652BCA014A15C41C8C2BC61CFF
:1006D0007D2BCB1C6E2BCB014B159A2B4B1D732BFB
:1006E000CB01CB159A2BCB1D782BCB014B169A2B1C
:1006F0004B1E9A2BCB01CB149A2B4B1D822BCB017B
:100700004B169A2BCB1D872BCB014B169A2B4B1ECE
:100710009A2BCB01CB149A2BCB1C912BCB014B15D5
:100720009A2B4B1D962BCB01CB159A2B4B1E9A2B3C
:10073000CB014B15441DC12B461DB22BCC1CA32B4A
:10074000CC014C15CF2B4C1DA82BCC01CC15CF2B9D
:10075000CC1DAD2BCC014C16CF2B4C1ECF2BCC017E
:10076000CC14CF2B4C1DB72BCC014C16CF2BCC1D52
:10077000BC2BCC014C16CF2B4C1ECF2BCC01CC1458
:10078000CF2BCC1CC62BCC014C15CF2B4C1DCB2B0F
:10079000CC01CC15CF2B4C1ECF2BCC014C15C41D3E
:1007A000F72BC61DE82BCD1CD92BCD014D155F13A2
:1007B000052C4D1DDE2BCD01CD15052CCD1DE32BBC
:1007C000CD014D16052C4D1E052CCD01CD14052C4B
:1007D0004D1DED2BCD014D16052CCD1DF22BCD0160
:1007E0004D16052C4D1E052CCD01CD14052CCD1C10
:1007F000FC2BCD014D15052C4D1D012CCD01CD152A
:10080000052C4D1E052CCD014D155F1B2E2C441EB5
:100810002E2C461E1F2CCE1C102CCE014E153C2C0F
:100820004E1D152CCE01CE153C2CCE1D1A2CCE0102
:100830004E163C2C4E1E3C2CCE01CE143C2C4E1D94
:10084000242CCE014E163C2CCE1D292CCE014E164A
:100850003C2C4E1E3C2CCE01CE143C2CCE1C332CFA
:10086000CE014E153C2C4E1D382CCE01CE153C2C05
:100870004E1E3C2CCE014E15C41E632CC61E542C9D
:10088000CF1C452CCF014F15712C4F1D4A2CCF0189
:10089000CF15712CCF1D4F2CCF014F16712C4F1E31
:1008A000712CCF01CF14712C4F1D592CCF014F1635
:1008B000712CCF1D5E2CCF014F16712C4F1E712C49
:1008C000CF01CF14712CCF1C682CCF014F15712C88
:1008D0004F1D6D2CCF01CF15712C4F1E712CCF01E8
:1008E0004F15DF189A2C451E9A2C471E8B2CD01CB6
:1008F0007C2CD0015015A82C501D812CD001D01576
:10090000A82CD01D862CD0015016A82C501EA82C27
:10091000D001D014A82C501D902CD0015016A82C1A
:10092000D01D952CD0015016A82C501EA82CD001FB
:10093000D014A82CD01C9F2CD0015015A82C501DD1
:10094000A42CD001D015A82C501EA82CD0015015D5
:10095000DF18D12CC51ED12CC71EC22CD11CB32C24
:10096000D1015115DF2C511DB82CD101D115DF2C2F
:10097000D11DBD2CD1015116DF2C511EDF2CD10110
:10098000D114DF2C511DC72CD1015116DF2CD11DE4
:10099000CC2CD1015116DF2C511EDF2CD101D114EA
:1009A000DF2CD11CD62CD1015115DF2C511DDB2C95
:1009B000D101D115DF2C511EDF2CD1015115DF18CB
:1009C000092D451F092D471FFA2CD21CEB2CD201F3
:1009D0005215DF13172D521DF02CD201D215172DF1
:1009E000D21DF52CD2015216172D521E172DD201F1
:1009F000D214172D521DFF2CD2015216172DD21DC5
:100A0000042DD2015216172D521E172DD201D214C9
:100A1000172DD21C0E2DD2015215172D521D132D3C
:100A2000D201D215172D521E172DD2015215DF18E3
:100A3000422DDF1B422DC51F422DC71F332DD31C56
:100A4000242DD3015315502D531D292DD301D3151A
:100A5000502DD31D2E2DD3015316502D531E502D26
:100A6000D301D314502D531D382DD3015316502DBF
:100A7000D31D3D2DD3015316502D531E502DD301A0
:100A8000D314502DD31C472DD3015315502D531D76
:100A90004C2DD301D315502D531E502DD30153157A
:100AA000B7214008C4004108C5005F18DF145F1C6F
:100AB000DF104808C9000C304A05031D05120C3030
:100AC0004B05031D85120C304C05031D05100C3021
:100AD0004D05031D85100C304E05031D87100C308D
:100AE0004F05031D07110C305005031D07100C3076
:100AF0005105031D87120C305205031D07120C30DF
:100B00005305031D871149080E020318B32D123037
:100B10004A05031D051612304B05031D85161230BC
:100B20004C05031D051412304D05031D85141230AC
:100B30004E05031D871412304F05031D0715123093
:100B40005005031D071412305105031D871612307E
:100B50005205031D071612305305031D8715FF307C
:100B60004802031908008F08031D08008720490860
:100B70000E02031CB32D18304A05031D0512063062
:100B80004A05031D051618304B05031D8512063056
:100B90004B05031D851618304C05031D0510063046
:100BA0004C05031D051418304D05031D8510063036
:100BB0004D05031D851418304E05031D87100630A2
:100BC0004E05031D871418304F05031D071106300D
:100BD0004F05031D071518305005031D071006307B
:100BE0005005031D071418305105031D87120630E8
:100BF0005105031D871618305205031D07120630D4
:100C00005205031D071618305305031D87110630C2
:080C10005305031D87150800C0
:084000000100030006000900A5
:02400E00CC33B1
:10420000010078007A007C007E007B0079007F004E
:104210007D007A0078007E007C007D007F007900C0
:104220000200F200F600FA00FE00F200F600FA00CA
:10423000FE00F200F600FA00FE00F200F600FA00BE
:10424000FF00050005000500050009000900090040
:1042500009000D000D000D000D00110011001100EE
:104260000100FF00FF00FF00FF00FF00FF00FF0054
:10427000FF00FF00FF00FF00FF00FF00FF00FF0046
:10428000FF007B00FF00FF00FF00FF00FF00FF00BA
:10429000FF00FF00FF00FF00FF00FF00FF00FF0026
:1042A000FF00FE00FF00FF00FF00FF00FF00FF0017
:1042B000FF00FF00FF00FF00FF00FF00FF00FF0006
:1042C000FF001100FF00FF00FF00FF00FF00FF00E4
:1042D000FF00FF00FF00FF00FF00FF00FF00FF00E6
:1042E000FF00FF00FF00FF00FF00FF00FF00FF00D6
:1042F000FF00FF00FF00FF00FF00FF00FF00DD00E8
:00000001FF
